:020000020000FC
:1000000086CD0000000000001FC0A4C18DC000000C
:10001000000097C00000000000000000020304067A
:10002000080C10182030406080000406080C1018DE
:100030002030406080A0C0000003070F1F000505AE
:100040000D050305030302004FB662FD0CC05520E9
:1000500041F00994C52DC095089483FDC795C4BD92
:1000600064604FBE1895C0916400089483FDC795E5
:10007000C4BD6B7FC0916400CF3F09F41EC070FF08
:100080001AC082FD05C04FBE939894989598189514
:1000900076FD0EC064FD0CC0C091B100C0FD929809
:1000A000C1FDC298C2FDC198CAEFC095CA95F1F7CB
:1000B0009398949895984FBE189524BCCC27C0640B
:1000C000C8BF6460F8CFC6CF70FFC4CF64FDC2CF95
:1000D000939AC0CF70FFBECF64FDBCCF949ABACFC5
:1000E00070FFB8CF64FDB6CF959AB4CF929A70FFE7
:1000F000B1CF64FDAFCFC7E0CA95F1F7939AAACF0D
:10010000C29A70FFA7CF64FDA5CFC7E0CA95F1F7EB
:10011000949AA0CFC19A70FF9DCF64FD9BCFC7E09A
:10012000CA95F1F7959A96CF4FB6C9B7CF7EC9BF9A
:100130006E7FCCB5CE0DDDB5DF1DDBBDCABD4FBEBC
:1001400018953FB68F7EA9B7A072A2118061A9B79A
:10015000AF7DA9BFA9B7AE7FA9BF7894A091680071
:10016000AA2341F085FD2FC0A0916800AA95A09315
:10017000680029C040E050E085FD15C0A6B396FD9B
:10018000A095A0FD4FEFAEB5A06496FDAF7BAEBDD0
:10019000AA27A062A8BF8D7FA6B396FDA095A0FD5B
:1001A0005FEF451739F7A8E161FDA093680085FD71
:1001B00003C0A8E1A09368004093960081604423A7
:1001C00011F02092990085FD0EC0A0916900AA232C
:1001D00031F0A0916900AA95A093690004C08061E4
:1001E000AA27A062A8BF80FF3DC0A09196004A2F19
:1001F00061FF8E7F85FD18C0403F08F040EFA42FBF
:10020000A295AF704A0F5091B600533069F0A69591
:10021000A69550FD01C0A69552FD03C0A41B4A2F10
:1002200003C04A0F08F44FEFA0919F004A1708F44B
:100230004A2F40936100A72FA670A1F073FD12C052
:10024000A0917000AA0FAA0F50919E005695569546
:10025000541708F0452F4A0F4093610018F4AFEF90
:10026000A0936100A0916100A0936300409163009E
:10027000A0919B004A1708F04A2F542EA091A0008D
:10028000AA2309F422C0542F5A1B10F4A42F50E0C3
:10029000BA2E8894AA1FAA2EA091A200A095AA22E5
:1002A000A50E58F0A091A100A21509F0AA95AA0EDA
:1002B000A093A10048F04A2D08C0A091A100BA1651
:1002C00008F0A395A093A1004FEF409364007F7BBB
:1002D000485F08F07064A0916000A395A09360004F
:1002E00059F0F894A9B7A160A9BF84FF03C0A9B7CA
:1002F000A062A9BF3FBE1895A0917400A395A093DA
:10030000740041E050916800552329F085FF03C037
:100310005A9550936800A0919600A13018F0209251
:1003200099000DC020929A002092A300A0919900FC
:10033000AF5FA093990018F0AFEFA0939900F894E5
:10034000A9B7A160A9BF84FF03C0A9B7A062A9BFD4
:100350003FBE18953FB646B557B58F7EA9B7A07278
:10036000A2118061A9B7AF7DA9BFA9B7AE7FA9BF10
:10037000789481FD25C0AEB5AF7B96FDA064AEBD7F
:100380008260A6B396FDA095A0FF05C040936500CE
:100390005093660041C1AEB5A06496FDAF7BAEBD83
:1003A000AA27A062A8BF8D7F85FF01C028C140E0B9
:1003B000A6B396FDA095A0FD22C14093960011C161
:1003C000AEB5A06496FDAF7BAEBD8D7F61FF72C000
:1003D000AEB5AF7B96FDA064AEBDAA27A062A8BF54
:1003E00082604093910050939200A0908F004A1930
:1003F000B09090005B09BB24A22C4C38520518F435
:100400002092950049C0A091D400AA2359F1483CFC
:10041000520528F4A0E1BA2EAAE0AA2E23C048363D
:10042000A1E05A0728F4A8E0BA2EAFE0AA2E1AC01D
:10043000403DA2E05A0728F4A4E0BA2EAEE1AA2E6D
:1004400011C0403AA5E05A0728F4A2E0BA2EACE366
:10045000AA2E08C04839A8E05A0720F4A1E0BA2E15
:10046000A8E7AA2EC42EA0919300CA1AD52EA09157
:100470009400DA0ADD202AF4AFEFC094D094CA1AAF
:10048000DA0A20929500A8E0A210A0E0CA14DA06C9
:1004900018F4A1E0A093950040939300509394002A
:1004A000409191005091920040938F0050939000A2
:1004B00042E097C0A09165004A1BA09166005A0BCC
:1004C00094FD82C093FD80C092FD7CC086FF03C076
:1004D000D52EC42E0CC05695479591FD73C05695E8
:1004E000479590FD6FC0D52EC42ED694C79461FD5C
:1004F00019C0AC2DAC51AD2DA24008F005C0DD20D7
:1005000089F4AC2DA85C70F4A0916700A395AA2390
:1005100011F0A0936700AA3008F471C020929600F1
:1005200081606DC0A0916700AA2319F0AA95A093DD
:100530006700A22C5091BA0097FD06C0A090C80099
:10054000533011F4A090D000AAEFAA0EA22DA21D44
:10055000CA18DA0A4FB74170533049F4442321F0E6
:1005600087FD05C0806803C087FF01C08F774423E3
:1005700059F0533031F4AFEFC094D094CA1ADA0A6C
:1005800003C040E050E020C0533049F4CC0CDD1CE7
:10059000AAE0CA1AD20818F4A0E0CA2ED22CAFEFF3
:1005A000CA16D20418F04FEF50E00EC0A091AC0074
:1005B000CA9E412D000C441F50E008F012C04FEFBE
:1005C00050E00FC05695479594FF07C0552309F09A
:1005D0004FEFA42FA6954A0F521D4F3F520508F02A
:1005E0004FEF40939600816061FF09C0AFE1A09595
:1005F000A923AB299A2F8F7DBB2009F48062A8E143
:10060000A093680085FF03C0AAE0A093680061FD85
:1006100003C085FD01C08F7E85FD03C0A6E0A093C9
:100620006900F894A9B7A160A9BF84FF03C0A9B766
:10063000A062A9BF3FBE189511E00AC013E008C030
:100640001AE006C01EE104C014E602C018EC00C0A7
:1006500005E1BB27BA95F1F70A95D9F71A95C1F7C5
:1006600008952AE338E709C020E33CE806C02AE2FF
:1006700034EB03C025E238EC00C0B091AD00BA9570
:1006800009F4089512E0BB27C29ABA95F1F7949A3B
:10069000BA95F1F79498BA95F1F7C298BA95F1F72F
:1006A000123009F0939A123009F4959AB091AD0086
:1006B000BA95F1F7123009F09398123009F4959831
:1006C000B7E8BA95F1F71A95F1F6022FB22FBA955D
:1006D000F1F70A95D9F73A9581F6C29A0895221B47
:1006E00039E0001F3A9509F40895221F211B18F4E0
:1006F000210F8894F6CF0894F4CF622C722CB0E0CE
:100700008894B395221F331FE0F737952795889477
:10071000912E802E020B130B10F4192D082D10F4BE
:10072000889401C00894661C771CBA9571F7172D40
:10073000062D0895322D11232AF43A95009510952F
:10074000031B130BF894029F712C002D129F912C08
:10075000802C7894780C172D921C292DB4E06B2EE8
:100760002695179507956A94D9F7332321F00095BC
:100770001095031B130B0895089510917B00169597
:1007800000917A000795B0917E00B01B0B2FB091BD
:100790007F00B10B1B2F28F40038BFEF1B0740F080
:1007A00009C00F37120508F405C00FE710E002C0BA
:1007B00000E81FEF009383001093840008950091D8
:1007C0008300B09180000B0F10918400B0918100E4
:1007D0001B1F20E03091840033230AF42A95B09146
:1007E00082002B1F1AF4203F40F00AC02F3008F47B
:1007F00007C00FEF1FEF2FE003C000E010E020EF75
:1008000030916300B0919B003B1718F4323030F008
:1008100009C0B0918400BB235AF004C0B091840099
:10082000BB2332F400938000109381002093820058
:1008300008952091D70000918300000F109184004B
:10084000111F78DF11232AF40038BFEF1B0740F097
:1008500009C00F37120508F405C00FE710E002C009
:1008600000E81FEF002352F0B0916200B01B0B2F85
:1008700018F0013008F00AC001E008C000950F5FD1
:10088000B09162000B0F08F001C00FEF00938500DC
:1008900008952091D80000918100109182004ADFD4
:1008A00011232AF40130BFEF1B0740F009C00F3FAE
:1008B000120508F405C00FEF10E002C001E01FEFC1
:1008C000112352F0B0918500B01B0B2F18F00130AE
:1008D00008F00AC001E008C000950F5FB0918500E4
:1008E0000B0F08F001C00FEF0093630008950FEFA6
:1008F00071FD1EC0B091D300BB23D1F0B0917B003D
:10090000BB23B1F00FEF10917B00E9DEF894B091BA
:10091000730072FDB5E00B9F112D002D789411230B
:1009200009F00FEFB0919E000B1710F400919E009C
:1009300000939D00089500917A0010917B0000546F
:100940001140B0919D0010F4BA9501C0B39511F01B
:10095000B0939D00089500C008952091B500B6B1F0
:10096000B6FDFBCF04B115B1B6B1BF77B6B9B09142
:10097000AA00B395B093AA00B83060F12092AA0003
:10098000B091D200BB2321F1112329F0B091AB002B
:10099000BF3F61F009C0B091AB000B1739F020F4F4
:1009A000BB2321F0BA9502C0B395E1F300919B00FF
:1009B000B093AB00B93B50F400ECBA3A38F400E81D
:1009C000BB3920F400E4BC3808F400E000939B003D
:1009D0007F7E0895B0919B00B39511F0B0939B007A
:1009E000B091AA00B73009F47061089502E3F89459
:1009F000B091D9000B9F012D000C001F7894B0918D
:100A00009B000B1710F000919B0000936100009376
:100A10006300502E0093640000939E00089520927E
:100A20007A00B0EFB0937B000895F8940CB51DB533
:100A30002091740078943091750060907600009356
:100A4000750010937600031B160971FD03C077FD36
:100A500080C028C070907700209377002709222358
:100A600019F00FEF1FEF0EC0809078009090790082
:100A700030937800609279000091750010917600B3
:100A80000819190920917A0030917B003695279535
:100A9000020F131F10F40FEF1FEF00937A00109353
:100AA0007B002BC020917A0030917B003901B4E0AB
:100AB0008B2EB2E09B2E343040F08A949A943830DA
:100AC00020F072FD02C08A949A94769467948A9476
:100AD000E1F726193709992021F0169507959A9480
:100AE000E1F7200F311F20937A0030937B0028F428
:100AF0003FEF30937A0030937B00323008F4706817
:100B000071FF02C0B3E00DC0B091C400009171004C
:100B1000023838F0B395003A08F0B395B63008F0D3
:100B2000B5E09B2EB4E08B2E10917B0000917A00F3
:100B300024E0169507952A95E1F70819120928F07F
:100B4000B02FB250B12FB20910F402E010E09801BA
:100B500026C020917A0030917B0039017694679409
:100B60006694669466942619320906950695200FB8
:100B7000321D20937A0030937B00323008F07F776B
:100B800004E0369527953695279526952695201BC2
:100B900010F0223008F422E089019090C40060FD3A
:100BA000FECFE0908B00F0908C006160B9B7B0612F
:100BB000B9BF380177FD41C07694679400938B00EC
:100BC00010938C00B92DB330E1F0B0FD04C0060DD8
:100BD000171D930106C0000F111F0250120922E0D9
:100BE00030E0B92DB33068F020938D0030938E0043
:100BF00000938700109388006092890070928A00A9
:100C00003AC000938D0010938E002093870030939C
:100C100088006092890070928A0071FF0DC0BFE069
:100C2000B0938D0020928E00B093890020928A00AC
:100C3000B0938B0020928C001EC0669400938B00B2
:100C4000B92DB33091F0B0FD03C0060D262D03C0C1
:100C5000000F025022E0B92DB33038F020938D0000
:100C6000009387006092890006C000938D00209356
:100C700087006092890000917C0002FD03500130E2
:100C800049F495FD12C0B0B7B860B0BFB0E0B06C29
:100C9000B7B90EC0023039F4B0B7B860B0BFB1E038
:100CA000B06CB7B905C095FDEECFB0B7B77FB0BF98
:100CB0000091A200000F10F4BBE60B270093A200E6
:100CC00060FDFECFB2E0B0936E006160B9B7B06175
:100CD000B9BFB72FB670D1F020917A0030917B0068
:100CE000369527953695279571FF02C0B0E43B0FE6
:100CF000F8940CB51DB5020F131F1BBD0ABD616032
:100D0000B0E1B8BFB9B7B061B9BF78940895686071
:100D100020927D0020E066FD20E206C068602092FF
:100D20007D0020E266FD20E001E011E077FD11C0CA
:100D3000B72FB67009F0677F14E100917B0006952C
:100D400009F403950F3008F00FE071FF02C004E1D1
:100D500014E160FD0FC0B0917D00BB2359F071FF1D
:100D600006C0B0916E00BA95B0936E0011F4706237
:100D700051C0ABDFB0B73B2FB77FB0BFB8B1B0B792
:100D800033FDB860B0BFB0917D00B395B0937D00E6
:100D9000B8B177FD06C0B1E071FDB3E0BA95F1F7E7
:100DA000B8B1B072B21709F02AC071FF05C003953F
:100DB000011708F00A95CDCF63FD05C00395011713
:100DC00008F0B2CFC6CF677FF8943CB56DB4709091
:100DD0007A00B0917B00770CBB1F08F4BFEF770C53
:100DE000BB1F08F4BFEF370D6B1E6BBC3ABD6160D3
:100DF000B0E1B8BFB9B7B061B9BF789495CFB09141
:100E00006D00B13008F490CF63FD8ECF0A9509F0E4
:100E1000A0CF7F7D20918D0030918E00F894B0E1BD
:100E2000B8BF0CB51DB5020F131F1BBD0ABDE09066
:100E30008700F09088006160B9B7B061B9BF78945D
:100E4000B72FB67039F0B0916D0072FFB395B093C3
:100E50006D0009C075FF07C066FD05C063FD03C0D6
:100E6000BF91BF9108C5089500E063FF01C001E094
:100E7000F89410917100B7E01B9F212D102D7894EC
:100E8000200F26951795269517952695179510935B
:100E90007100183718F4B8E7B09371000091710031
:100EA000B09172000B1720F0606193989498959818
:100EB00060FDFECFE0908900F0908A006160B9B7D4
:100EC000B061B9BF0895AC98B2E095FD0AC0F8943E
:100ED000B0937C00C29A929862FF01C0959A789470
:100EE000F9C0F894B0937C00C29AC19862FF01C027
:100EF000939A7894EFC0AC9AB3E082FF24C095FD3A
:100F000011C002E0F894B0937C00E0E8F0E00093B8
:100F1000B1009598C19A62FF02C0949A01C0C2982C
:100F20007894D8C002E0F894B0937C00E0E8F0E058
:100F30000093B1009398929A62FF02C0949A01C004
:100F4000C2987894C7C095FD0BC0F894B0937C000C
:100F5000EAE6F0E0959862FF01C0949A7894BAC0EE
:100F6000F894B0937C00EAE6F0E0939862FF01C049
:100F7000949A7894AFC0AC98B4E095FD0AC0F89408
:100F8000B0937C00929AC19862FF01C0949A7894C1
:100F9000A1C0F894B0937C00C19A929862FF01C0FE
:100FA000949A789497C0AC9AB5E082FF24C095FDDE
:100FB00011C001E0F894B0937C00E6E7F0E0009304
:100FC000B1009498C29A62FF02C0939A01C09298AD
:100FD000789480C004E0F894B0937C00EAE8F0E0F4
:100FE0000093B1009498C29A62FF02C0959A01C022
:100FF000C19878946FC095FD0BC0F894B0937C00B5
:10100000E4E6F0E0949862FF01C0939A789462C09D
:10101000F894B0937C00E0E7F0E0949862FF01C0A0
:10102000959A789457C0AC98B6E095FD0AC0F894AC
:10103000B0937C00C19AC29862FF01C0939A7894E1
:1010400049C0F894B0937C00929AC29862FF01C0A4
:10105000959A78943FC0AC9AB1E082FF24C095FD88
:1010600011C004E0F894B0937C00EAE8F0E000934B
:10107000B1009398929A62FF02C0959A01C0C198FC
:10108000789428C001E0F894B0937C00E6E7F0E0A3
:101090000093B1009598C19A62FF02C0939A01C073
:1010A0009298789417C095FD0BC0F894B0937C008B
:1010B000E0E7F0E0939862FF01C0959A78940AC047
:1010C000F894B0937C00E4E6F0E0959862FF01C0EC
:1010D000939A78946F7E089523E630E0F901209288
:1010E000B100939894989598929AC29AC19A6B7FFE
:1010F0000895A2EBB0E00FEF0D930D930D930D93B8
:1011000003E00D9304E00D930AE00D9303E00D93CB
:1011100001E00D9301E00D93AEEBB0E001E00D9323
:101120000FEF0D930D930D930D930D9303E00D931E
:101130000FEF0D930FEF0D930D9305E20D9300ED5F
:101140000D930AEF0D930AEF0D9304E00D930FEF4B
:101150000D9301E00D9300E00D930AE70D930FEF5F
:101160000D9300E00D9301E00D9300E00D9303E07B
:101170000D9300E00D9308952091B9008B7F2330EB
:1011800009F48460B091BA00B33019F09F7DB1FDCD
:1011900090629F7BB091BB00B1FD9064223011F052
:1011A000886001C0877F08950A95E00FF21DB49111
:1011B0000895ECE1F0E00091B200F6DFB093D700C3
:1011C000ECE1F0E00091B300EFDFB093D800EAE289
:1011D000F0E00091B800E8DFB093D9000091B800CA
:1011E000023008F402E000937300B091CE000FEFDC
:1011F000B23009F400EAB33009F402E80093720057
:10120000E8E3F0E00091D500CFDFB093A0000895AF
:1012100008952091C8003091C900B091BA00B33050
:1012200009F43E5097FF02C020E03FEFB32FB21BFE
:101230006B2EB25810F4B2E86B2E00E00395609E5E
:10124000B12DBD57D8F30093AC0008959068E1DF4D
:10125000F9D9F8D920E030E0B0E16B2EEFD9B091A8
:1012600096002B0F321D6A94C9F7B4E03695279586
:10127000BA95E1F7822E9F77CCDF0895F894E3E0EA
:10128000F0E0B9E0B7BFB491B078C1F3F894A89595
:10129000B1B5B861B1BDB0E0B1BDB4E0BEBFBFE5AE
:1012A000BDBF1ADFB6E0B8BBB6E1B7BBB8E0B5BBAF
:1012B000BCE1B4BBB4E0B2BBBCE3B1BB2224A0E050
:1012C000B0E02D92AA31E9F7A0E6B0E00FEF2D9241
:1012D0000A95E9F7B1E0B093A2000BDF08D3B7E0BD
:1012E000B06CB7B9B6B1B460B068B6B90091CA0015
:1012F0000093AD00B1E0B0936A00F894A7D9B1D9DA
:10130000A1D9B2D99FD9B3D99DD978D39FD99ED924
:101310009BD9F8940AEF1AEFA6B396FDA095A0FF0B
:101320001FC01A95C9F70A95B1F7E0E0FCE1B59145
:10133000B43E39F4B591B03E21F4B591BF3F09F404
:101340000CC0E0E0F395F395B591B83F49F4B59141
:10135000B43931F4B591BA3A19F4EE27F6950994F7
:101360000BDF27DF55DF55DF0091CA000093AD008A
:10137000B3DEB2E0B3BFB2E0BEBDB2E0B5BDB1E531
:10138000B8BFB9BFB0B70B2FB77FB0BFB8B1B0B758
:1013900003FDB860B0BF50D97894DDDA20927000B8
:1013A000BEB5B06496FDBF7BBEBDB9B7B062B9BF74
:1013B000BB27B062B8BF8D7F49D9626033E02CE0B3
:1013C000B0919500BB2321F42CE03A9509F4A1CF0C
:1013D00039D980FF9ECF8E7FB0919600B23078F3DE
:1013E000B92FBF710091980000939700B0939800B7
:1013F000B01729F72A9521F76D7FBEB5B06496FD29
:10140000BF7BBEBDBB27B062B8BF8D7FB091D4009B
:10141000BB2321F48062B92FB0709B2F8F7B209269
:10142000670012D985FF05C0B0916700BA3008F097
:10143000806404D902E085FF01C000E0B09196000D
:10144000B017B8F3F8940DD90CD90BD97894FED80D
:1014500020928600B091BA00B33009F47EC0EED875
:10146000B091BE00B13008F478C0B0916A00B130DC
:1014700008F473C085FD18C0B0919600BF3F08F412
:101480006CC0F894F7D87894DFD8B0919600B1305A
:10149000C0F7F894E6D8D4D8E4D87894D5D8B091E9
:1014A0009600BF3FB0F3DCC2B8E09B2E9068F89482
:1014B000B0DE7894C9D8F8949F77ABDE8090960020
:1014C000B0919600BF37789408F44FC0B5D8F8941F
:1014D000D1D878949A9451F7B9DEB82DB550B0931D
:1014E000C900B4D8F8948FD27894BAE09B2E906853
:1014F000F8948FDE7894A8D8F8949F778ADE80904D
:101500009600B0919600BF37789478F795D8F89404
:10151000A8D896D8A6D878949A9449F797DEB82D8B
:10152000BB5FB093C8000B2F1091C900125810F088
:10153000100B20F4B2E80B0F0093C90087D8F89481
:1015400003D270D2789480D8F89463DE7894B09106
:101550009600BF3F08F48ECF83C200919600B091F1
:1015600086000B1710F0009386006ED801E0B09152
:10157000BA00B35009F405E0B0919600B01708F036
:1015800069CFF89477D876D875D878945FD82092B8
:101590006A0020926B0020926C00B0916B00B395B2
:1015A000B0936B00BF3F71F5B0916C00B395B093F1
:1015B0006C00B091CC0009E1BA9559F002E3BA95FC
:1015C00041F00DE7BA9529F00AEFBA9511F0209293
:1015D0006C00B0916C00B017A8F07EDD2DD8B091F2
:1015E0006C00BA95B0936C0020926B00B091CB0068
:1015F000B093AD00F8943ED87894B091CA00B093FF
:10160000AD0022D81DD8B0916800BB2319F485FF26
:1016100001C07FCE01E085FD01C006E0B0919600DB
:10162000B01708F4BACFB091BA00B35009F00CD893
:10163000B0916800BB2309F46CCEF8944DDD209284
:1016400061002092620020926300522C209264007C
:101650002092A1007894B091B700BB0FB0939F0087
:1016600020927E0020927F002092800020928100B4
:10167000209282002092AA0060E070E02092710027
:10168000B8E0B093AA007061D7D7B7E074FDB6E0B8
:10169000B06CB7B9B6B1B068B064B6B9B6B1B6FDA2
:1016A000FDCF04B115B1B6B1BF77B6B9112309F0BA
:1016B0000FEF0093AB0051D9B8E0B093AA0070616E
:1016C0005BDDF894BFEFB0939B0090D9B0916100BF
:1016D000B0939B00B0939C00B0939D007894B1E0D0
:1016E000B0936100B09363005B2EB0936400B0933D
:1016F000A400B0919A00B093A300B091BA00B330A7
:1017000019F49F7D87FD90627160726020926D0078
:101710008ADCA1DC84D989D982D987D980D9FEDA3B
:101720002BD8A2DBD0DB81D9F2DA65FD26D877FF92
:10173000DED877FD00D998DBDEDB77D9EFDA65FDFF
:101740003ED892DB18DC71D9E2DA65FD72D88CDB09
:101750002ADC6BD9E3DA65FD9CD886DB64DC65D9CD
:10176000D6DAB7E074FDB6E0B06CB7B9B6B1B06820
:10177000B064B6B979DB6FDC58D9EFD871FF21C0FE
:10178000B0919E00B0939B00B0939C00B0919A00E2
:10179000B093A300B1E0B093A40018E12CE0B091A5
:1017A0006D00B11740F07D7F746020936F00BFEF34
:1017B000B0939B0006C0B0919600B13008F0AFCF57
:1017C00064C072FF15C066FD13C0B0916F00BA957A
:1017D00019F47B7F7860A3CFB0936F00B09196002F
:1017E000B13008F09CCFB091BA00B33009F04DC0D1
:1017F00020927000B091990002E81091D600112358
:1018000009F003E0B01708F040C085FF04C0B091B4
:101810006800BB23D1F1B091BA00B33081F495FDDB
:1018200003C087FD04C00BC087FF01C008C066FD70
:1018300006C06064B0919E00B0939B0085CF00EF1E
:1018400066FF05C0B0919E00B0939B0000E2B0918E
:101850007B00B01708F463CF66FF17C06F7B9F7DD6
:1018600087FD90627460B2E1B0936F00B0919E000A
:10187000B0939B0054CFB0917000B395B0937000BB
:10188000B0919600BB2309F002C020927000F8943A
:1018900023DC8090B900B2E0B093B9006DDC809297
:1018A000B900209261002092620020926300522CC5
:1018B0002092640020929F0060E070E07894C4D68B
:1018C0000BDC0091D600002319F0939A949A959A14
:1018D000B7E0B06CB7B9B6B1B460B068B6B985FF5F
:1018E00005C0B0917000B43008F013CD52CEEDE0D9
:1018F000F0E023D00A3509F01BC0EEE0F0E01DD087
:10190000053A09F015C03AE0A2EBB0E0E3E0F0E000
:1019100014D00D9331963A95D9F739E1AEEBB0E09A
:10192000EFE0F0E00AD00D9331963A95D9F702C076
:10193000E0DB0AD0E8E2F0E00895E199FECFEEBBEB
:10194000FFBBE09A0DB308951ED03AE0A2EBB0E0E1
:10195000E3E0F0E00D910FD031963A95D9F739E1F7
:10196000AEEBB0E0EFE0F0E00D9105D031963A95A6
:10197000D9F712D00895E199FECF0DBBEEBBFFBBA6
:10198000E29AE19A0895EDE0F0E00FEFF4DFEEE087
:10199000F0E00FEFF0DF0895EDE0F0E00AE5EBDFB7
:1019A000EEE0F0E005EAE7DF08953091AE00009147
:1019B000AF00313011F40093B600323011F40093CF
:1019C000B700333011F40093B800343011F40093B1
:1019D000C400353011F40093B900363011F400938F
:1019E000D500373011F40093CE00383011F4009355
:1019F000BA00393011F40093BB00089525E026D6D3
:101A00002A95E9F708952DD62FD631D633D618D694
:101A100028D62AD62CD62ED613D623D625D627D6E8
:101A200029D6089527D623D61FD61BD609D622D667
:101A30001ED61AD616D604D61DD619D615D611D648
:101A400008958090AE009090AF000BD60AD609D6CC
:101A5000F7D58A94D1F70ED6F3D59A94E1F7089585
:101A6000F894D1DF7894CADFC9DFB1E0B093AE005B
:101A7000B1E0B093AF002092B000F894E2DF789428
:101A8000B5E06B2E70909600E1D5B09196007B1674
:101A9000C9F7B13018F0BF3F40F107C086DFF894B6
:101AA00053DFB1DFB8E0B1BDA9DF6A9459F7B09157
:101AB000B000B395B093B000B33008F4DECF9EDF32
:101AC000B091AF00B395B093AF00F894B091AE0071
:101AD000BA95EEE3F0E0EB0FF21D049178940395D4
:101AE000B091AF00B01708F4C6CF88DF87DFB091A0
:101AF000AE00B395B093AE00B091AE00BA3008F42A
:101B0000B7CFF7DAF89420DFB8E0B1BD77DFB6CB16
:00000001FF
